:02000000912944
:08000800FF00030E8312031335
:10001000A0000A0EA100040EA2008A110A1294295F
:100020008316981683120C1E12282E0899000800B9
:10003000AF01B001B101FF30B200B301B4012E0A2B
:10004000031D24280130B3001816B408031D3B28F3
:100050008C1E2D280230B4002528B308031D252846
:10006000AE08031D36280130B4002528AF03AF08C1
:100070000319AE0325283408023A031D4B28181D26
:1000800044281A08B1004B28981C49281812181641
:100090004B281A08B2003208B5000800C830831295
:1000A0000313AE0018203508A4002803031D5D28A3
:1000B0002408A7000230A80008002408A600013088
:1000C000A8000330AB00080083120313AB08031928
:1000D000E1282B08033A031D7B280230AB00DF30F8
:1000E000831607058700DF3083120705AE00203036
:1000F0002E048700E1282B08023A031DD72801307F
:10010000AB0027082506031DE1282608123A031D27
:10011000A228F330831607058700F3308312070502
:10012000AE0004302E0487009630A300FE30831604
:1001300008058800FE3083120805AE0001302E0449
:100140008800E12826081C3A031DBF28F3308316D7
:1001500007058700F33083120705AE0008302E0430
:1001600087009630A300FD30831608058800FD3017
:1001700083120805AE0002302E048800E12826080C
:100180001E3A031DE128FB30831608058800FB306A
:1001900083120805AE0004302E0488009630A300B8
:1001A0002908AE0010202A08AE001020E128DF3018
:1001B000831607058700DF308312070587000130AB
:1001C000AB00A308031DF528F3308316070587004D
:1001D000F330831207058700F8308316080588007E
:1001E000F83083120805880008002303A3000800E4
:1001F000DF308316031307058700DF3083120705FE
:100200008700FD30831607058700FD308312070540
:100210008700FD30831607058700FD308312070530
:10022000AC0002302C048700F330831607058700EA
:10023000F3308312070587000130A800AB01831655
:1002400081120116F03001058312AC0006302C0437
:10025000831681008B178B169030831298008B17B2
:1002600083168C1608000430831603139F000508BC
:100270008312AC000130831605048500813083129F
:100280009F00AD0128302D0203184829AD0A4229EC
:1002900004301F049F001F194B292C08831685006A
:1002A00007309F00803083129F00080083120313E1
:1002B0001E08AC0008000730831603139F000430AB
:1002C000980081309900831298019817C0308316E6
:1002D0008100F82017308316060486001730831239
:1002E0000605A5000F3C03187C290F302505AC003E
:1002F00008302C04A5007F290F302505A5002030EB
:10030000831606048600203083120605AC00AA017D
:1003100020302C020319AA0A332156212C08A900E7
:100320006A298A110A125B290B1D982964200B1176
:10033000831203138C1E9E294E208C12220E8400E1
:0E034000210E8A00200E8300FF0E7F0E0900A2
:02400E003A3D39
:00000001FF
